:020000040000FA
:0408000049EF0BF0C1
:1008100003B276EF05F0F2B494EF05F09EB09CEFD2
:1008200005F09EB2A4EF05F0F2A81AEF04F0F2B2C0
:1008300025EF04F0F2A620EF04F0F2B022EF04F06E
:10084000F8EF0AF0F296F290FF00CD90F2929EA09F
:100850002FEF04F00101533F2FEF04F0542BAEC1F2
:10086000B2F1AFC1B3F1B0C1B4F1B1C1B5F1AAC138
:10087000AEF1ABC1AFF1ACC1B0F1ADC1B1F1A6C148
:10088000AAF1A7C1ABF1A8C1ACF1A9C1ADF1A2C158
:10089000A6F1A3C1A7F1A4C1A8F1A5C1A9F19EC168
:1008A000A2F19FC1A3F1A0C1A4F1A1C1A5F19AC178
:1008B0009EF19BC19FF19CC1A0F19DC1A1F196C188
:1008C0009AF197C19BF198C19CF199C19DF1CECF4E
:1008D00096F1CFCF97F153C198F154C199F1CF6AF6
:1008E000CE6A0101536B546B9E90CD800FBC0F8E6E
:1008F0000FBA7EEF04F00F8AF8EF0AF00F8C0FBEEC
:10090000BAEF04F096C19AF197C19BF198C19CF19E
:1009100099C19DF19AC19EF19BC19FF19CC1A0F12B
:100920009DC1A1F19EC1A2F19FC1A3F1A0C1A4F1FB
:10093000A1C1A5F1A2C1A6F1A3C1A7F1A4C1A8F1CB
:10094000A5C1A9F1A6C1AAF1A7C1ABF1A8C1ACF19B
:10095000A9C1ADF1AAC1AEF1ABC1AFF1ACC1B0F16B
:10096000ADC1B1F1AEC1B2F1AFC1B3F1B0C1B4F13B
:10097000B1C1B5F101015E6B5F6B606B616B96514C
:100980005E2797515F2398516023995161239A51B3
:100990005E279B515F239C5160239D5161239E5193
:1009A0005E279F515F23A0516023A1516123A25173
:1009B0005E27A3515F23A4516023A5516123A65153
:1009C0005E27A7515F23A8516023A9516123AA5133
:1009D0005E27AB515F23AC516023AD516123AE5113
:1009E0005E27AF515F23B0516023B1516123B251F3
:1009F0005E27B3515F23B4516023B5516123D89072
:100A00000101613360335F335E33D890010161339C
:100A100060335F335E33D8900101613360335F33FD
:100A20005E3300C10CF101C10DF102C10EF103C131
:100A30000FF104C110F105C111F106C112F107C196
:100A400013F108C114F109C115F10AC116F10BC166
:100A500017F134C135F111B839EF05F00101620E1B
:100A6000046F010E056F000E066F000E076F42EF58
:100A700005F00101A70E046F020E056F000E066F50
:100A8000000E076F5EC100F15FC101F160C102F1AC
:100A900061C103F1EDEC28F003BF04D018BE02D011
:100AA00018A0108C11A05AEF05F010BA5AEF05F0FB
:100AB0000F80108A0CC100F10DC101F10EC102F1CD
:100AC0000FC103F110C104F111C105F112C106F10A
:100AD00013C107F114C108F115C109F116C10AF1DA
:100AE00017C10BF135C134F1F8EF0AF00392ABB244
:100AF000AB98AB88030103EE00F080517F0BE92631
:100B000004C0EFFF802B8151805D700BD8A48B82D5
:100B100000008051815D700BD8A48B9281518019A7
:100B2000D8B40790F8EF0AF0F2940101453FF8EFCE
:100B30000AF0462BF8EF0AF09E900101533FF8EFC0
:100B40000AF0542BF8EF0AF09E9211B81FEF08F04C
:100B5000040062A1ACEF05F08BB4B6EF05F010AC69
:100B6000B6EF05F08B84109CB7EF05F08B94077CF3
:100B700007ACD2EF05F0C274C2B4CCEF05F0C3CF1E
:100B8000B3F5C4CFB4F50501D890B433B333D890DE
:100B9000B433B333D3EF05F0C3CF55F1C4CF56F11F
:100BA000D3EF05F0C28207B440EF06F047C14BF126
:100BB00048C14CF149C14DF14AC14EF15EC162F1EB
:100BC0005FC163F160C164F161C165F196C1B6F1C5
:100BD00097C1B7F198C1B8F199C1B9F19AC1BAF109
:100BE0009BC1BBF19CC1BCF19DC1BDF19EC1BEF1D9
:100BF0009FC1BFF1A0C1C0F1A1C1C1F1A2C1C2F1A9
:100C0000A3C1C3F1A4C1C4F1A5C1C5F1A6C1C6F178
:100C1000A7C1C7F1A8C1C8F1A9C1C9F1AAC1CAF148
:100C2000ABC1CBF1ACC1CCF1ADC1CDF1AEC1CEF118
:100C3000AFC1CFF1B0C1D0F1B1C1D1F1B2C1D2F1E8
:100C4000B3C1D3F1B4C1D4F1B5C1D5F1B3C5B5F5D4
:100C5000B4C5B6F5B5C5B7F5B6C5B8F5010155517A
:100C60005B2756515C23E86A5D230E2E40EF06F0A9
:100C70005CC157F15DC158F15B6B5C6B5D6B078EBE
:100C80000201002FF8EF0AF03C0E006F1950E00B44
:100C9000E00AE866128816AE108E00C10CF101C1A0
:100CA0000DF102C10EF103C10FF104C110F105C134
:100CB00011F106C112F107C113F108C114F109C104
:100CC00015F10AC116F10BC117F134C135F1050157
:100CD0002F51000AD8B418EF07F005012F51010A6F
:100CE000D8B4A2EF06F005012F51020AD8B4E3EF01
:100CF00006F005012F51030AD8B4E3EF06F0050111
:100D00002F51040AD8B4E3EF06F005012F51050A6C
:100D1000D8B4E3EF06F005012F51060AD8B4E3EF8B
:100D200006F005012F51070AD8B4E3EF06F00501DC
:100D30002F51320AD8B4A0EF06F02F6B18EF07F04E
:100D400018EF07F005015367ADEF06F05467ADEFFC
:100D500006F05567ADEF06F05667B1EF06F018EFF5
:100D600007F057C500F158C501F159C502F15AC540
:100D700003F10101010E046F000E056F000E066FF6
:100D8000000E076FEDEC28F000C157F501C158F5D2
:100D900002C159F503C15AF50067D6EF06F00167A5
:100DA000D6EF06F00267D6EF06F0036718EF07F0FC
:100DB00053C557F554C558F555C559F556C55AF597
:100DC0000F8818EF07F005013067E9EF06F018EF1C
:100DD00007F00FBEFEEF06F010A003EF07F00101D1
:100DE0004767FAEF06F04867FAEF06F04967FAEF4F
:100DF00006F04A67FEEF06F003EF07F007AE03EFD9
:100E000007F015EF07F00501312F18EF07F03C0E42
:100E1000316F302F18EF07F00101000E626FE00E06
:100E2000636FA50E646F010E656F0501306B0F884F
:100E30000501626B33B71EEF07F062810CC100F150
:100E40000DC101F10EC102F10FC103F110C104F196
:100E500011C105F112C106F113C107F114C108F166
:100E600015C109F116C10AF117C10BF135C134F1F1
:100E700000C10CF101C10DF102C10EF103C10FF16E
:100E800004C110F105C111F106C112F107C113F13E
:100E900008C114F109C115F10AC116F10BC117F10E
:100EA00034C135F101018A675DEF07F08B675DEFB3
:100EB00007F08C675DEF07F08D6761EF07F091EF4A
:100EC00007F08EC100F18FC101F190C102F191C113
:100ED00003F10101010E046F000E056F000E066F95
:100EE000000E076FEDEC28F000C18EF101C18FF10B
:100EF00002C190F103C191F1006786EF07F001672D
:100F000086EF07F0026786EF07F0036791EF07F0BF
:100F10008AC18EF18BC18FF18CC190F18DC191F19D
:100F20000F80D57ED5BE6DD0D6CF47F1D7CF48F153
:100F300045C149F1E86AE8CF4AF118BE02D018A0CD
:100F4000108C109047C100F148C101F149C102F174
:100F50004AC103F101010A0E046F000E056F000E75
:100F6000066F000E076FEDEC28F003AF1080010153
:100F700054A7C7EF07F00F9A0F9C0F9E0101000EB8
:100F80005E6F600E5F6F3D0E606F080E616F010156
:100F900047BFD7EF07F04867D7EF07F04967D7EFAC
:100FA00007F04A67D7EF07F0F288FCEF07F0F298F6
:100FB0005E6B5F6B606B616B966B976B986B996BFD
:100FC0009A6B9B6B9C6B9D6B9E6B9F6BA06BA16BDD
:100FD000A26BA36BA46BA56BA66BA76BA86BA96B8D
:100FE000AA6BAB6BAC6BAD6BAE6BAF6BB06BB16B3D
:100FF000B26BB36BB46BB56BD76AD66A0101456B44
:10100000466B0CC100F10DC101F10EC102F10FC11F
:1010100003F110C104F111C105F112C106F113C1B0
:1010200007F114C108F115C109F116C10AF117C180
:101030000BF135C134F1F8EF0AF0F8EF0AF00201D4
:10104000002F61EF0AF0D59ED6CF47F1D7CF48F1F8
:1010500045C149F1E86AE8CF4AF1D76AD66A010189
:10106000456B466BD58E1950E00BE00AE866128896
:1010700017AE108E16AE1B8C00C10CF101C10DF124
:1010800002C10EF103C10FF104C110F105C111F14C
:1010900006C112F107C113F108C114F109C115F11C
:1010A0000AC116F10BC117F134C135F10FA0109A26
:1010B00011B866EF08F00101620E046F010E056FB2
:1010C000000E066F000E076F6FEF08F00101A70E0C
:1010D000046F020E056F000E066F000E076F47C10A
:1010E00000F148C101F149C102F14AC103F1EDEC3F
:1010F00028F003BF82EF08F018BE02D018A0108CB1
:1011000011B00F800CC100F10DC101F10EC102F14F
:101110000FC103F110C104F111C105F112C106F1B3
:1011200013C107F114C108F115C109F116C10AF183
:1011300017C10BF135C134F102013C0E006F00C143
:101140000CF101C10DF102C10EF103C10FF104C197
:1011500010F105C111F106C112F107C113F108C167
:1011600014F109C115F10AC116F10BC117F134C10F
:1011700035F105012F51000AD8B46AEF09F00501D5
:101180002F51010AD8B4F4EF08F005012F51020ADB
:10119000D8B435EF09F005012F51030AD8B435EF63
:1011A00009F005012F51040AD8B435EF09F0050103
:1011B0002F51050AD8B435EF09F005012F51060A61
:1011C000D8B435EF09F005012F51070AD8B435EF2F
:1011D00009F005012F51320AD8B4F2EF08F02F6B55
:1011E0006AEF09F06AEF09F005015367FFEF08F0B5
:1011F0005467FFEF08F05567FFEF08F0566703EFFD
:1012000009F06AEF09F057C500F158C501F159C559
:1012100002F15AC503F10101010E046F000E056FC2
:10122000000E066F000E076FEDEC28F000C157F5B9
:1012300001C158F502C159F503C15AF5006728EFFD
:1012400009F0016728EF09F0026728EF09F003674A
:101250006AEF09F053C557F554C558F555C559F50A
:1012600056C55AF50F886AEF09F0050130673BEF64
:1012700009F06AEF09F00FBE50EF09F010A055EF2A
:1012800009F0010147674CEF09F048674CEF09F09E
:1012900049674CEF09F04A6750EF09F055EF09F044
:1012A00007AE55EF09F067EF09F00501312F6AEF3E
:1012B00009F03C0E316F302F6AEF09F00101000E8A
:1012C000626FE00E636FA50E646F010E656F05011E
:1012D000306B0F880501626B33B770EF09F06281E4
:1012E0000CC100F10DC101F10EC102F10FC103F1FA
:1012F00010C104F111C105F112C106F113C107F1CA
:1013000014C108F115C109F116C10AF117C10BF199
:1013100035C134F100C10CF101C10DF102C10EF172
:1013200003C10FF104C110F105C111F106C112F1A1
:1013300007C113F108C114F109C115F10AC116F171
:101340000BC117F134C135F101018A67AFEF09F024
:101350008B67AFEF09F08C67AFEF09F08D67B3EFE4
:1013600009F0E3EF09F08EC100F18FC101F190C1E6
:1013700002F191C103F10101010E046F000E056F2E
:10138000000E066F000E076FEDEC28F000C18EF125
:1013900001C18FF102C190F103C191F10067D8EF53
:1013A00009F00167D8EF09F00267D8EF09F0036789
:1013B000E3EF09F08AC18EF18BC18FF18CC190F1FE
:1013C0008DC191F10F80109047C100F148C101F12A
:1013D00049C102F14AC103F101010A0E046F000E76
:1013E000056F000E066F000E076FEDEC28F003AFDF
:1013F0001080010154A709EF0AF00F9A0F9C0F9E6D
:101400000101000E5E6F600E5F6F3D0E606F080E93
:10141000616F47C100F148C101F149C102F14AC100
:1014200003F10101140E046F050E056F000E066F27
:10143000000E076FEDEC28F003AF22EF0AF0F28800
:1014400047EF0AF0F2985E6B5F6B606B616B966BB7
:10145000976B986B996B9A6B9B6B9C6B9D6B9E6B60
:101460009F6BA06BA16BA26BA36BA46BA56BA66B10
:10147000A76BA86BA96BAA6BAB6BAC6BAD6BAE6BC0
:10148000AF6BB06BB16BB26BB36BB46BB56B0CC1C4
:1014900000F10DC101F10EC102F10FC103F110C144
:1014A00004F111C105F112C106F113C107F114C114
:1014B00008F115C109F116C10AF117C10BF135C1C7
:1014C00034F104008BB46CEF0AF010AC6CEF0AF04E
:1014D0008B84109C6DEF0AF08B94077C07AC88EF2F
:1014E0000AF0C274C2B482EF0AF0C3CFB3F5C4CF1E
:1014F000B4F50501D890B433B333D890B433B333D3
:1015000089EF0AF0C3CF55F1C4CF56F189EF0AF045
:10151000C28207B4F6EF0AF047C14BF148C14CF163
:1015200049C14DF14AC14EF15EC162F15FC163F143
:1015300060C164F161C165F196C1B6F197C1B7F1BF
:1015400098C1B8F199C1B9F19AC1BAF19BC1BBF187
:101550009CC1BCF19DC1BDF19EC1BEF19FC1BFF157
:10156000A0C1C0F1A1C1C1F1A2C1C2F1A3C1C3F127
:10157000A4C1C4F1A5C1C5F1A6C1C6F1A7C1C7F1F7
:10158000A8C1C8F1A9C1C9F1AAC1CAF1ABC1CBF1C7
:10159000ACC1CCF1ADC1CDF1AEC1CEF1AFC1CFF197
:1015A000B0C1D0F1B1C1D1F1B2C1D2F1B3C1D3F167
:1015B000B4C1D4F1B5C1D5F1B3C5B5F5B4C5B6F56F
:1015C000B5C5B7F5B6C5B8F5010155515B275651FC
:1015D0005C23E86A5D230E2EF6EF0AF05CC157F13A
:1015E0005DC158F15B6B5C6B5D6B078EF8EF0AF0C9
:1015F00002C0E0FF005001C0D8FF1000A6B2FEEF0D
:101600000AF00CC0A9FF0BC0A8FFA69EA69CA6844A
:10161000F29E550EA76EAA0EA76EA682F28EA69413
:10162000A6B210EF0BF00C2A1200A96EA69EA69C83
:10163000A680A8500C2A120004012C0E826F57ECD1
:101640000EF0E8EC29F00C5015EC0BF0E8CF00F1AF
:101650000C5015EC0BF0E8CF01F101AF35EF0BF0BA
:101660000101FF0E026FFF0E036F8BEC29F029675B
:1016700041EF0BF00401200E826F57EC0EF046EFA5
:101680000BF004012D0E826F57EC0EF0B5EC27F035
:101690001200076A0F6A106A116A126A0F010D0EB2
:1016A000C16E860EC06E030EC26E0F01680E896E8B
:1016B000130E926E080E8A6EF30E936E8B6A900E66
:1016C000946EC80E15EC0BF0E8CFE8FF1098E8A078
:1016D000108810A805D00E0E216E8E0E226E04D03A
:1016E0000F0E216E8F0E226E67EC2AF0F18EF19EA6
:1016F000FC0E15EC0BF0E8CF0BF00BA011800BA249
:1017000011820BA411840BA81188C90E15EC0BF0E3
:10171000E8CF16F0CA0E15EC0BF0E8CF17F0CB0EA1
:1017200015EC0BF0E8CF18F0CC0E15EC0BF0E8CF71
:1017300019F01B6A1C6A0E6A01015B6B5C6B5D6BC6
:10174000576B586BF29A0101476B486B496B4A6BB8
:101750004B6B4C6B4D6B4E6B4F6B506B516B526BBD
:10176000456B466BD76AD66A0F01280ED56EF28A92
:101770009D90B00ECD6E01015E6B5F6B606B616B17
:10178000626B636B646B656B666B676B686B696BD5
:10179000536B546BCF6ACE6A0F9A0F9C0F9E9D803D
:1017A000760ECA6E9D8202013C0E006FCC6A160E48
:1017B00015EC0BF0E8CF00F1170E15EC0BF0E8CFAD
:1017C00001F1180E15EC0BF0E8CF02F1190E15EC33
:1017D0000BF0E8CF03F1010103AF09EF0CF0E8ECE7
:1017E00029F0160E0C6E00C10BF0FEEC0AF0170E7D
:1017F0000C6E01C10BF0FEEC0AF0180E0C6E02C16B
:101800000BF0FEEC0AF0190E0C6E03C10BF0FEECAF
:101810000AF000C18AF101C18BF102C18CF103C150
:101820008DF100C18EF101C18FF102C190F103C1B0
:1018300091F11A0E15EC0BF0E8CF00F11B0E15EC30
:101840000BF0E8CF01F11C0E15EC0BF0E8CF02F124
:101850001D0E15EC0BF0E8CF03F1010103AF5FEFB4
:101860000CF0E8EC29F01A0E0C6E00C10BF0FEEC47
:101870000AF01B0E0C6E01C10BF0FEEC0AF01C0E00
:101880000C6E02C10BF0FEEC0AF01D0E0C6E03C1D3
:101890000BF0FEEC0AF01A0E15EC0BF0E8CF00F19D
:1018A0001B0E15EC0BF0E8CF01F11C0E15EC0BF044
:1018B000E8CF02F11D0E15EC0BF0E8CF03F100C1EB
:1018C00092F101C193F102C194F103C195F1240E8B
:1018D000AC6E900EAB6E240EAC6E080EB86E000EA1
:1018E000B06E1F0EAF6E0401806B816B0F01900E06
:1018F000AB6E0F019D8A0301806B816BC26B8B9273
:10190000EFEC2EF0EFEC2EF04BEC30F0CEEC2CF0B8
:10191000200E15EC0BF0E8CF2FF505012F51FF0A33
:10192000D8A49AEF0CF02F6B200E0C6E2FC50BF085
:10193000FEEC0AF00501010E306F3C0E316F250EF2
:1019400015EC0BF0E8CF00F1260E15EC0BF0E8CF0C
:1019500001F1270E15EC0BF0E8CF02F1280E15EC83
:101960000BF0E8CF03F1010103AFD1EF0CF0E8EC8D
:1019700029F0250E0C6E00C10BF0FEEC0AF0260ECD
:101980000C6E01C10BF0FEEC0AF0270E0C6E02C1CA
:101990000BF0FEEC0AF0280E0C6E03C10BF0FEEC0F
:1019A0000AF000C153F501C154F502C155F503C158
:1019B00056F500C157F501C158F502C159F503C1EB
:1019C0005AF5290E15EC0BF0E8CF5BF505015C51DB
:1019D0005B5DD8A05BC55CF505012F51020A0EE1E5
:1019E00081B8FEEF0CF005015C2FFBEF0CF05BC53E
:1019F0005CF5FEEF0CF081BA8AEF30F0210E15ECA9
:101A00000BF0E8CF00F1220E15EC0BF0E8CF01F15E
:101A1000230E15EC0BF0E8CF02F1240E15EC0BF0C1
:101A2000E8CF03F1010103AF44EF0DF0E8EC29F03A
:101A3000210E0C6E00C10BF0FEEC0AF0220E0C6EB3
:101A400001C10BF0FEEC0AF0230E0C6E02C10BF08C
:101A5000FEEC0AF0240E0C6E03C10BF0FEEC0AF053
:101A6000210E15EC0BF0E8CF00F1220E15EC0BF077
:101A7000E8CF01F1230E15EC0BF0E8CF02F1240EB4
:101A800015EC0BF0E8CF03F100C15DF501C15EF587
:101A900002C15FF503C160F516EC2CF018EC2BF0D9
:101AA00070EC2AF005012F51030A12E005012F51B5
:101AB000040A1DE005012F51050A24E005012F51FC
:101AC000060A32E005012F51070A38E0A7EF0DF0B2
:101AD000ACC500F101010F0E001701010051000A11
:101AE00036E001010051050A32E0A4EF0DF0ACC56B
:101AF00000F101010F0E001701010051000A27E05B
:101B0000A4EF0DF00501AC51000A21E00501AC5134
:101B1000150A1DE00501AC51300A19E00501AC5170
:101B2000450A15E0A4EF0DF00501AC51000A0FE0E5
:101B30000501AC51300A0BE0A4EF0DF00501AC51EA
:101B4000000A05E0A4EF0DF081BA8AEF30F00790AB
:101B50000001F28EF28C07B039EF26F00FB0E6EFFD
:101B60001FF010BEE6EF1FF012B8E6EF1FF00FB83F
:101B700089EF19F00301805181197F0BD8B439EF37
:101B800026F013EE00F081517F0BE126812BE7CF89
:101B9000E8FFE00BD8B439EF26F023EE82F0C25113
:101BA0003F0BD926E7CFDFFFC22BDF50780AD8A43E
:101BB00039EF26F007808EC100F18FC101F190C18D
:101BC00002F191C103F10101040E046F000E056FD3
:101BD000000E066F000E076FEDEC28F000AFFAEF75
:101BE0000DF00101030E8E6F000E8F6F000E906FCF
:101BF000000E916F03018251720AD8B4D1EF1FF029
:101C00008251520AD8B4D1EF1FF08251750AD8B46C
:101C1000D1EF1FF08251630AD8B4F3EF22F0825162
:101C2000690AD8B480EF1CF082517A0AD8B493EFD5
:101C30001DF08251490AD8B41FEF1CF08251500A9E
:101C4000D8B43DEF1BF08251700AD8B480EF1BF07E
:101C50008251540AD8B4ABEF1BF08251740AD8B445
:101C6000F1EF1BF08251410AD8B46BEF0EF08251B4
:101C70006D0AD8B44FEF12F082514D0AD8B468EF14
:101C800012F08251730AD8B401EF1FF08251530A47
:101C9000D8B466EF1FF082514C0AD8B4F7EF12F0B7
:101CA0008251590AD8B4A0EF11F02AEF23F00401B1
:101CB00014EE00F080517F0BE12682C4E7FF802BF9
:101CC000120004010D0E826F57EC0EF00A0E826FA7
:101CD00057EC0EF012000401410E826F57EC0EF02B
:101CE00003018351310AD8B4C0EF10F003018351CE
:101CF000320AD8B416EF10F003018351330AD8B476
:101D00009FEF0FF003018351340AD8B48FEF0EF028
:101D100004013F0E826F57EC0EF028EF23F0CC0E3B
:101D200015EC0BF0E8CF0BF004012C0E826F57EC92
:101D30000EF003018451310AD8B4B3EF0EF0030161
:101D40008451300AD8B4B5EF0EF0030184514D0A26
:101D5000D8B4BFEF0EF003018451540AD8B4C6EFD3
:101D60000EF0DDEF0EF08A8401D08A940BAE04D021
:101D70000BAC02D00BBA21D0E00E0B1218D01F0E04
:101D80000B168539E844E00B0B1211D0E00E0B1650
:101D900029EC2AF085C332F186C333F10101296BA6
:101DA00036EC2AF0ADEC29F000511F0B0B12CC0ED3
:101DB0000C6E0BC00BF0FEEC0AF00401340E826FC7
:101DC00057EC0EF004012C0E826F57EC0EF0CC0E87
:101DD00015EC0BF0E8CF19F08AB406D00401300EF0
:101DE000826F57EC0EF005D00401310E826F57EC74
:101DF0000EF004012C0E826F57EC0EF01938E840FB
:101E0000070BE8CF82F40401300E822757EC0EF066
:101E100004012C0E826F57EC0EF0E8EC29F01950FB
:101E20001F0BE8CF00F18BEC29F032C182F40401E2
:101E3000300E822757EC0EF033C182F40401300ECD
:101E4000822757EC0EF004012C0E826F57EC0EF037
:101E5000E8EC29F02CC000F100AF0BD0FF0E016FB1
:101E6000FF0E026FFF0E036F04012D0E826F57EC01
:101E70000EF08BEC29F031C182F40401300E822780
:101E800057EC0EF032C182F40401300E822757EC79
:101E90000EF033C182F40401300E822757EC0EF0AD
:101EA00004012C0E826F57EC0EF0E8EC29F02BC0E9
:101EB00000F18BEC29F031C182F40401300E82274D
:101EC00057EC0EF032C182F40401300E822757EC39
:101ED0000EF033C182F40401300E822757EC0EF06D
:101EE00004012C0E826F57EC0EF0E8EC29F02DC0A7
:101EF00000F100AF0BD0FF0E016FFF0E026FFF0E5F
:101F0000036F04012D0E826F57EC0EF08BEC29F05D
:101F100031C182F40401300E822757EC0EF032C139
:101F200082F40401300E822757EC0EF033C182F4A4
:101F30000401300E822757EC0EF028EF23F0CB0E71
:101F400015EC0BF0E8CF0BF004012C0E826F57EC70
:101F50000EF003018451450AD8B4C3EF0FF003011A
:101F60008451440AD8B4C6EF0FF003018451300AFB
:101F7000D8B4C9EF0FF003018451310AD8B4CDEFC2
:101F80000FF0D8EF0FF00B9ED2EF0FF00B8ED2EFC9
:101F90000FF0FC0E0B16D2EF0FF0FC0E0B160B80A1
:101FA000D2EF0FF0CB0E0C6E0BC00BF0FEEC0AF074
:101FB0000401330E826F57EC0EF004012C0E826F79
:101FC00057EC0EF0CB0E15EC0BF0E8CF18F018BE66
:101FD000F1EF0FF00401450E826F57EC0EF0F6EFB3
:101FE0000FF00401440E826F57EC0EF004012C0E2A
:101FF000826F57EC0EF00401300E826F57EC0EF03A
:1020000004012C0E826F57EC0EF018B00FEF10F099
:102010000401300E826F57EC0EF014EF10F0040143
:10202000310E826F57EC0EF028EF23F0CA0E15EC3C
:102030000BF0E8CF0BF004012C0E826F57EC0EF082
:1020400003018451450AD8B446EF10F003018451CE
:10205000440AD8B449EF10F0030184514D0AD8B4B2
:1020600052EF10F003018451410AD8B44CEF10F044
:1020700003018451460AD8B44FEF10F00301845194
:10208000560AD8B45AEF10F06BEF10F00B9E65EFC4
:1020900010F00B8E65EF10F00B9C65EF10F00B8CC1
:1020A00065EF10F0F80E0B1685C3E8FF070B0B1257
:1020B00065EF10F0C70E0B1685C3E8FF070BE84667
:1020C000E846E8460B1265EF10F0CA0E0C6E0BC026
:1020D0000BF0FEEC0AF0CA0E15EC0BF0E8CF17F08F
:1020E0000401320E826F57EC0EF004012C0E826F49
:1020F00057EC0EF017BE84EF10F00401450E826F0E
:1021000057EC0EF089EF10F00401440E826F57EC8B
:102110000EF004012C0E826F57EC0EF017C0E8FF92
:10212000070BE8CF82F40401300E822757EC0EF043
:1021300004012C0E826F57EC0EF017BCA7EF10F0C5
:102140000401410E826F57EC0EF0ACEF10F0040169
:10215000460E826F57EC0EF004012C0E826F57EC86
:102160000EF017C0E8FF380BE842E842E842E8CF3B
:1021700082F40401300E822757EC0EF028EF23F092
:10218000C90E15EC0BF0E8CF0BF004012C0E826F9A
:1021900057EC0EF003018451450AD8B4DEEF10F07D
:1021A00003018451440AD8B4E1EF10F003018451D3
:1021B0004D0AD8B4E4EF10F0F2EF10F00B9EECEF04
:1021C00010F00B8EECEF10F0F80E0B1685C3E8FF45
:1021D000070B0B12ECEF10F0C90E0C6E0BC00BF0DE
:1021E000FEEC0AF00401310E826F57EC0EF0040190
:1021F0002C0E826F57EC0EF0C90E15EC0BF0E8CFE9
:1022000016F016BE06D00401450E826F57EC0EF094
:1022100005D00401440E826F57EC0EF004012C0E21
:10222000826F57EC0EF016C0E8FF070BE8CF82F480
:102230000401300E822757EC0EF004012C0E826F41
:1022400057EC0EF00780E8EC29F027C0E8FF003BD0
:1022500000430043030B8BEC29F033C182F40401EB
:10226000300E822757EC0EF004012C0E826F57ECD3
:102270000EF0E8EC29F027C001F1019F019D28C074
:1022800000F101018BEC29F02FC182F40401300E22
:10229000822757EC0EF030C182F40401300E822701
:1022A00057EC0EF031C182F40401300E822757EC56
:1022B0000EF032C182F40401300E822757EC0EF08A
:1022C00033C182F40401300E822757EC0EF0040172
:1022D0002C0E826F57EC0EF0E8EC29F029C001F1CA
:1022E0002AC000F1D89001330033D8900133003375
:1022F00001018BEC29F02FC182F40401300E8227FA
:1023000057EC0EF030C182F40401300E822757ECF6
:102310000EF031C182F40401300E822757EC0EF02A
:1023200032C182F40401300E822757EC0EF033C123
:1023300082F40401300E822757EC0EF028EF23F0D0
:10234000FC0E15EC0BF0E8CF0BF003018351520AA1
:10235000D8B4D7EF11F003018351720AD8B4DAEF81
:1023600011F003018351500AD8B4DDEF11F00301DD
:102370008351700AD8B4E0EF11F003018351550A7C
:10238000D8B4E3EF11F003018351750AD8B4E6EF36
:1023900011F003018351430AD8B4EFEF11F00301A8
:1023A0008351630AD8B4F2EF11F0FBEF11F00B90F8
:1023B000F5EF11F00B80F5EF11F00B92F5EF11F046
:1023C0000B82F5EF11F00B94F5EF11F00B84F5EFA4
:1023D00011F00B96F5EF11F00B86F5EF11F00B985D
:1023E000F5EF11F00B88F5EF11F0FC0E0C6E0BC041
:1023F0000BF0FEEC0AF00401590E826F57EC0EF060
:102400001190119211941198FC0E15EC0BF0E8CF7D
:102410000BF00BA011800BA211820BA411840BA84E
:10242000118811A01BEF12F00401520E826F57ECBD
:102430000EF020EF12F00401720E826F57EC0EF0D6
:1024400011A82AEF12F00401430E826F57EC0EF030
:102450002FEF12F00401630E826F57EC0EF011A201
:1024600039EF12F00401500E826F57EC0EF03EEF80
:1024700012F00401700E826F57EC0EF011A448EFB9
:1024800012F00401550E826F57EC0EF04DEF12F072
:102490000401750E826F57EC0EF028EF23F0040153
:1024A0006D0E826F57EC0EF003018351300AD8B4E1
:1024B000A7EF12F003018351310AD8B4BAEF12F03A
:1024C00003018351320AD8B4CDEF12F02AEF23F082
:1024D00004014D0E826F57EC0EF029EC2AF084C3F4
:1024E00031F185C332F186C333F10101296B36EC3A
:1024F0002AF0ADEC29F003018351300AD8B48FEFF4
:1025000012F003018351310AD8B497EF12F003019E
:102510008351320AD8B49FEF12F02AEF23F0FD0E58
:102520000C6E00C10BF0FEEC0AF0A7EF12F0FE0EED
:102530000C6E00C10BF0FEEC0AF0BAEF12F0FF0EC9
:102540000C6E00C10BF0FEEC0AF0CDEF12F00401AE
:10255000300E826F57EC0EF004012C0E826F57EC98
:102560000EF0E8EC29F0FD0E15EC0BF0E8CF00F1D1
:10257000DEEF12F00401310E826F57EC0EF0040111
:102580002C0E826F57EC0EF0E8EC29F0FE0E15ECE5
:102590000BF0E8CF00F1DEEF12F00401320E826F93
:1025A00057EC0EF0E8EC29F004012C0E826F57EC8A
:1025B0000EF0FF0E15EC0BF0E8CF00F18BEC29F0DC
:1025C00031C182F40401300E822757EC0EF032C183
:1025D00082F40401300E822757EC0EF033C182F4EE
:1025E0000401300E822757EC0EF028EF23F0030190
:1025F0008351300AD8B462EF16F003018351310AD7
:10260000D8B48FEF17F003018351320AD8B4FDEF2D
:1026100017F003018351330AD8B40DEF18F003010A
:102620008351340AD8B41DEF18F003018351350AE1
:10263000D8B48EEF19F003018351360AD8B4BCEF39
:1026400019F003018351370AD8B4C4EF15F0030120
:102650008351460AD8B4E2EF18F0030183514D0AC2
:10266000D8B43DEF14F0030183516D0AD8B457EF8D
:1026700014F0030183515A0AD8B409EF17F003018B
:102680008351490AD8B4BCEF1AF003018351500AB0
:10269000D8B4EEEF19F003018351540AD8B467EFB0
:1026A0001AF003018351630AD8B477EF14F00301E1
:1026B0008351430AD8B46FEF15F003018351730AB5
:1026C000D8B475EF14F003018351610AD8B48AEFCE
:1026D00013F003018351650AD8B4B2EF16F0030179
:1026E0008351450AD8B4C0EF16F003018351620A42
:1026F000D8B4CEEF16F003018351420AD8B4DCEF10
:1027000016F003018351760AD8B4EAEF16F0D8A484
:102710002AEF23F004014C0E826F57EC0EF00401F7
:10272000610E826F57EC0EF018EC2BF004012C0EAA
:10273000826F57EC0EF0E8EC29F0ABC500F1010117
:102740008BEC29F031C182F40401300E822757EC62
:102750000EF032C182F40401300E822757EC0EF0E5
:1027600033C182F40401300E822757EC0EF00401CD
:102770002C0E826F57EC0EF0E8EC29F0ACC500F19E
:1027800001018BEC29F031C182F40401300E822763
:1027900057EC0EF032C182F40401300E822757EC60
:1027A0000EF033C182F40401300E822757EC0EF094
:1027B00004012C0E826F57EC0EF0E8EC29F0ADC549
:1027C00000F101018BEC29F031C182F40401300EDB
:1027D000822757EC0EF032C182F40401300E8227BA
:1027E00057EC0EF033C182F40401300E822757EC0F
:1027F0000EF004012C0E826F57EC0EF0E8EC29F07D
:10280000AEC500F101018BEC29F031C182F4040165
:10281000300E822757EC0EF032C182F40401300EE4
:10282000822757EC0EF033C182F40401300E822768
:1028300057EC0EF004012C0E826F57EC0EF0E8EC12
:1028400029F0B2C500F101018BEC29F031C182F40D
:102850000401300E822757EC0EF032C182F40401DD
:10286000300E822757EC0EF033C182F40401300E93
:10287000822757EC0EF0EAEF19F029EC2AF084C316
:1028800033F136EC2AF0ADEC29F0200E0C6E00C1CD
:102890000BF0FEEC0AF000C12FF505012F51000AE4
:1028A00006E005012F51010A02E0B2EC2BF0040111
:1028B0004C0E826F57EC0EF004014D0E826F57ECF8
:1028C0000EF004012C0E826F57EC0EF0E8EC29F0AC
:1028D0002FC500F18BEC29F033C182F40401300ED6
:1028E000822757EC0EF0EAEF19F08AEF30F004017E
:1028F0004C0E826F57EC0EF00401630E826F57ECA2
:102900000EF070EC2AF004012C0E826F57EC0EF0E2
:102910008CEC14F0EAEF19F0E8EC29F0B1C500F105
:102920000101003B0F0E00178BEC29F033C182F43C
:102930000401300E822757EC0EF0B1C500F1010101
:102940000F0E010100178BEC29F033C182F4040152
:10295000300E822757EC0EF004012D0E826F57ECDB
:102960000EF0B0C500F10101003B0F0E00178BEC1B
:1029700029F033C182F40401300E822757EC0EF0A7
:10298000B0C500F101010F0E010100178BEC29F019
:1029900033C182F40401300E822757EC0EF004019B
:1029A0002D0E826F57EC0EF0AFC500F10101003B18
:1029B0000F0E00178BEC29F033C182F40401300EA6
:1029C000822757EC0EF0AFC500F101010F0E010197
:1029D00000178BEC29F033C182F40401300E8227FA
:1029E00057EC0EF00401200E826F57EC0EF0AEC5CE
:1029F00000F10F0E010100178BEC29F033C182F4B6
:102A00000401300E822757EC0EF00401200E826F75
:102A100057EC0EF0ADC500F101010101003B0F0EB6
:102A200000178BEC29F033C182F40401300E8227A9
:102A300057EC0EF0ADC500F101010F0E01010017BA
:102A40008BEC29F033C182F40401300E822757EC5D
:102A50000EF004013A0E826F57EC0EF0ACC500F197
:102A60000101003B0F0E00178BEC29F033C182F4FB
:102A70000401300E822757EC0EF0ACC500F10101C5
:102A80000F0E010100178BEC29F033C182F4040111
:102A9000300E822757EC0EF004013A0E826F57EC8D
:102AA0000EF0ABC500F10101003B0F0E00178BECDF
:102AB00029F033C182F40401300E822757EC0EF066
:102AC000ABC500F101010F0E00178BEC29F033C1EB
:102AD00082F40401300E822757EC0EF0120084C3FA
:102AE000E8FF0F0BE83AE8CFB1F585C3E8FF0F0B1D
:102AF0000501B11387C3E8FF0F0BE83AE8CFB0F543
:102B000088C3E8FF0F0B0501B0138AC3E8FF0F0B62
:102B1000E83AE8CFAFF58BC3E8FF0F0B0501AF1321
:102B20008DC3E8FF0F0BE8CFAEF58FC3E8FF0F0BA7
:102B3000E83AE8CFADF590C3E8FF0F0B0501AD1300
:102B400092C3E8FF0F0BE83AE8CFACF593C3E8FF78
:102B50000F0B0501AC1395C3E8FF0F0BE83AE8CF64
:102B6000ABF596C3E8FF0F0B0501AB13CBEC2AF0D6
:102B700004014C0E826F57EC0EF00401430E826F7D
:102B800057EC0EF081EF14F0078404014C0E826FB5
:102B900057EC0EF00401370E826F57EC0EF0040173
:102BA0002C0E826F57EC0EF005012E51130A06E031
:102BB00005012E51170A0DE05FEF16F00101000E1E
:102BC000006F000E016F100E026F000E036FF2EF28
:102BD00015F00101000E006F000E016F000E026F74
:102BE000010E036F8BEC29F02AC182F40401300E30
:102BF000822757EC0EF02BC182F40401300E82279D
:102C000057EC0EF02CC182F40401300E822757ECF1
:102C10000EF02DC182F40401300E822757EC0EF025
:102C20002EC182F40401300E822757EC0EF02FC122
:102C300082F40401300E822757EC0EF030C182F48A
:102C40000401300E822757EC0EF031C182F40401EA
:102C5000300E822757EC0EF032C182F40401300EA0
:102C6000822757EC0EF033C182F40401300E822724
:102C700057EC0EF004012C0E826F57EC0EF00101A0
:102C8000100E006F000E016F000E026F000E036F3A
:102C90008BEC29F031C182F40401300E822757EC0D
:102CA0000EF032C182F40401300E822757EC0EF090
:102CB00033C182F40401300E822757EC0EF00794E2
:102CC000EAEF19F007844BEC30F0E8EC29F02DC561
:102CD00000F18BEC29F004014C0E826F57EC0EF0E2
:102CE0000401300E826F57EC0EF004012C0E826F3F
:102CF00057EC0EF031C182F40401300E822757ECFC
:102D00000EF032C182F40401300E822757EC0EF02F
:102D100033C182F40401300E822757EC0EF0040117
:102D20002C0E826F57EC0EF0E8EC29F02EC500F166
:102D30008BEC29F031C182F40401300E822757EC6C
:102D40000EF032C182F40401300E822757EC0EF0EF
:102D500033C182F40401300E822757EC0EF0079441
:102D6000EAEF19F004014C0E826F57EC0EF00401EB
:102D7000650E826F57EC0EF072EC2CF0EAEF19F052
:102D800004014C0E826F57EC0EF00401450E826F69
:102D900057EC0EF089EC2CF0EAEF19F004014C0E20
:102DA000826F57EC0EF00401620E826F57EC0EF04A
:102DB000B7EC2CF0EAEF19F004014C0E826F57ECDF
:102DC0000EF00401420E826F57EC0EF0A0EC2CF0D6
:102DD000EAEF19F004014C0E826F57EC0EF004017B
:102DE000760E826F57EC0EF004012C0E826F57ECBA
:102DF0000EF010A807D00401310E826F57EC0EF0D0
:102E0000EAEF19F00401300E826F57EC0EF0EAEF92
:102E100019F004014C0E826F57EC0EF004015A0EAB
:102E2000826F57EC0EF004012C0E826F57EC0EF0FF
:102E30004BEC30F0E8EC29F005012E51130A06E0C6
:102E400005012E51170A0DE03AEF17F00101000EAF
:102E5000006F000E016F100E026F000E036F3AEF4D
:102E600017F00101000E006F000E016F000E026FDF
:102E7000010E036F0101100E046F000E056F000EAE
:102E8000066F000E076F1EEC29F08BEC29F02AC1AB
:102E900082F40401300E822757EC0EF02BC182F42D
:102EA0000401300E822757EC0EF02CC182F404018D
:102EB000300E822757EC0EF02DC182F40401300E43
:102EC000822757EC0EF02EC182F40401300E8227C7
:102ED00057EC0EF02FC182F40401300E822757EC1C
:102EE0000EF030C182F40401300E822757EC0EF050
:102EF00031C182F40401300E822757EC0EF032C14A
:102F000082F40401300E822757EC0EF033C182F4B4
:102F10000401300E822757EC0EF0EAEF19F0078417
:102F200004014C0E826F57EC0EF00401310E826FDB
:102F300057EC0EF004012C0E826F57EC0EF025C5F5
:102F400000F126C501F127C502F128C503F10101F1
:102F5000100E046F000E056F000E066F000E076F57
:102F60001EEC29F08BEC29F02AC182F40401300E0A
:102F7000822757EC0EF02BC182F40401300E822719
:102F800057EC0EF02CC182F40401300E822757EC6E
:102F90000EF02DC182F40401300E822757EC0EF0A2
:102FA0002EC182F40401300E822757EC0EF02FC19F
:102FB00082F40401300E822757EC0EF030C182F407
:102FC0000401300E822757EC0EF031C182F4040167
:102FD000300E822757EC0EF032C182F40401300E1D
:102FE000822757EC0EF033C182F40401300E8227A1
:102FF00057EC0EF00794EAEF19F0078404014C0E29
:10300000826F57EC0EF00401320E826F57EC0EF017
:10301000A5EC2EF00794EAEF19F0078404014C0E9A
:10302000826F57EC0EF00401330E826F57EC0EF0F6
:1030300002EC2FF007949AEF17F0078404014C0E6E
:10304000826F57EC0EF00401340E826F57EC0EF0D5
:1030500004012C0E826F57EC0EF029EC2AF084C389
:103060002AF185C32BF186C32CF187C32DF188C3C8
:103070002EF189C32FF18AC330F18BC331F18CC398
:1030800032F18DC333F10101296B36EC2AF0ADEC3E
:1030900029F0100E046F000E056F000E066F000E73
:1030A000076FFEEC28F000C121F501C122F502C135
:1030B00023F503C124F5FEEC2FF034C5ABF535C57F
:1030C000ACF536C5ADF537C5AEF538C5AFF539C584
:1030D000B0F53AC5B1F58CEC14F004012C0E826FFA
:1030E00057EC0EF03BC500F13CC501F13DC502F1C6
:1030F0003EC503F10101000E046F000E056F010EC5
:10310000066F000E076F1EEC29F08BEC29F0296783
:103110008CEF18F091EF18F004012D0E826F57EC30
:103120000EF030C182F40401300E822757EC0EF00D
:1031300031C182F40401300E822757EC0EF00401F5
:103140002E0E826F57EC0EF032C182F40401300E65
:10315000822757EC0EF033C182F40401300E82272F
:1031600057EC0EF004012C0E826F57EC0EF0E8ECD9
:1031700029F03FC500F140C501F154EC24F00401F1
:103180002C0E826F57EC0EF0E8EC29F041C500F1EF
:103190008BEC29F031C182F40401300E822757EC08
:1031A0000EF032C182F40401300E822757EC0EF08B
:1031B00033C182F40401300E822757EC0EF00794DD
:1031C000EAEF19F029EC2AF085C32AF186C32BF126
:1031D00087C32CF188C32DF189C32EF18AC32FF147
:1031E0008BC330F18CC331F18DC332F18EC333F117
:1031F0000101296B36EC2AF0ADEC29F00101010E3A
:10320000046F000E056F000E066F000E076FEDECE9
:1032100028F0100E046F000E056F000E066F000EF2
:10322000076FFEEC28F000C129F501C12AF502C1A3
:103230002BF503C12CF52CEC2EF004014C0E826F03
:1032400057EC0EF00401460E826F57EC0EF00401AD
:103250002C0E826F57EC0EF025C500F126C501F14A
:1032600027C502F128C503F10101100E046F000EFD
:10327000056F000E066F000E076F1EEC29F08BEC39
:1032800029F02AC182F40401300E822757EC0EF097
:103290002BC182F40401300E822757EC0EF02CC1B2
:1032A00082F40401300E822757EC0EF02DC182F417
:1032B0000401300E822757EC0EF02EC182F4040177
:1032C000300E822757EC0EF02FC182F40401300E2D
:1032D000822757EC0EF030C182F40401300E8227B1
:1032E00057EC0EF031C182F40401300E822757EC06
:1032F0000EF032C182F40401300E822757EC0EF03A
:1033000033C182F40401300E822757EC0EF0EAEF4D
:1033100019F00F9802EC2FF02AEF23F004014C0E65
:10332000826F57EC0EF00401350E826F57EC0EF0F1
:1033300004012C0E826F57EC0EF0E8EC29F00784A4
:10334000B5C500F107948BEC29F031C182F404017A
:10335000300E822757EC0EF032C182F40401300E99
:10336000822757EC0EF033C182F40401300E82271D
:1033700057EC0EF0EAEF19F0C5EC2EF0E8EC29F06E
:1033800033C500F18BEC29F004014C0E826F57EC31
:103390000EF00401360E826F57EC0EF004012C0E75
:1033A000826F57EC0EF031C182F40401300E822797
:1033B00057EC0EF032C182F40401300E822757EC34
:1033C0000EF033C182F40401300E822757EC0EF068
:1033D000EAEF19F061EC0EF02AEF23F004014C0E35
:1033E000826F57EC0EF00401500E826F57EC0EF016
:1033F00004012C0E826F57EC0EF085C32AF186C3B0
:103400002BF187C32CF188C32DF189C32EF18AC318
:103410002FF18BC330F18CC331F18DC332F18EC3E8
:1034200033F1010136EC2AF0ADEC29F003018451AF
:10343000530A0DE0030184514D0A38E00401780E6F
:10344000826F57EC0EF061EC0EF02AEF23F00401CE
:10345000530E826F57EC0EF0250E0C6E00C10BF070
:10346000FEEC0AF0260E0C6E01C10BF0FEEC0AF029
:10347000270E0C6E02C10BF0FEEC0AF0280E0C6E4B
:1034800003C10BF0FEEC0AF000C153F501C154F585
:1034900002C155F503C156F500C157F501C158F5F4
:1034A00002C159F503C15AF5CBEF1AF004014D0ED4
:1034B000826F57EC0EF0290E0C6E00C10BF0FEEC83
:1034C0000AF000C15BF500C15CF5CBEF1AF0040116
:1034D0004C0E826F57EC0EF00401540E826F57ECC5
:1034E0000EF004012C0E826F57EC0EF084C32AF10B
:1034F00085C32BF186C32CF187C32DF188C32EF130
:1035000089C32FF18AC330F18BC331F18DC332F1FE
:103510008EC333F1010136EC2AF0ADEC29F0010144
:10352000000E046F000E056F010E066F000E076F90
:10353000FEEC28F0210E0C6E00C10BF0FEEC0AF040
:10354000220E0C6E01C10BF0FEEC0AF0230E0C6E85
:1035500002C10BF0FEEC0AF0240E0C6E03C10BF05E
:10356000FEEC0AF000C15DF501C15EF502C15FF538
:1035700003C160F5CBEF1AF004014C0E826F57ECDB
:103580000EF00401490E826F57EC0EF004012C0E70
:10359000826F57EC0EF0250E15EC0BF0E8CF00F122
:1035A000260E15EC0BF0E8CF01F1270E15EC0BF011
:1035B000E8CF02F1280E15EC0BF0E8CF03F18BEC0D
:1035C00029F06EEC27F00401730E826F57EC0EF0B9
:1035D00004012C0E826F57EC0EF0E8EC29F0290E56
:1035E00015EC0BF0E8CF00F18BEC29F06EEC27F036
:1035F0000401730E826F57EC0EF004012C0E826FE3
:1036000057EC0EF057C500F158C501F159C502F14C
:103610005AC503F18BEC29F06EEC27F00401730E10
:10362000826F57EC0EF004012C0E826F57EC0EF0F7
:10363000E8EC29F05CC500F18BEC29F06EEC27F08A
:1036400004016D0E826F57EC0EF004012C0E826F98
:1036500057EC0EF05DC500F15EC501F15FC502F1EA
:1036600060C503F145EC23F004012C0E826F57EC8A
:103670000EF061EC0EF02AEF23F083C32AF184C32D
:103680002BF185C32CF186C32DF187C32EF188C39E
:103690002FF189C330F18AC331F18BC332F18CC36E
:1036A00033F1010136EC2AF0ADEC29F0160E0C6E68
:1036B00000C10BF0FEEC0AF0170E0C6E01C10BF00E
:1036C000FEEC0AF0180E0C6E02C10BF0FEEC0AF0D4
:1036D000190E0C6E03C10BF0FEEC0AF000C18AF16A
:1036E00001C18BF102C18CF103C18DF100C18EF1DA
:1036F00001C18FF102C190F103C191F11FEF1CF0E4
:1037000083C32AF184C32BF185C32CF186C32DF129
:1037100087C32EF188C32FF189C330F18AC331F1F9
:103720008BC332F18CC333F1010136EC2AF0ADECDE
:1037300029F000C18AF101C18BF102C18CF103C1F2
:103740008DF100C18EF101C18FF102C190F103C171
:1037500091F11FEF1CF083C32AF184C32BF185C3C1
:103760002CF186C32DF187C32EF188C32FF189C3B5
:1037700030F18AC331F18CC332F18DC333F10101D1
:1037800036EC2AF0ADEC29F00101000E046F000EBA
:10379000056F010E066F000E076FFEEC28F01A0E83
:1037A0000C6E00C10BF0FEEC0AF01B0E0C6E01C19A
:1037B0000BF0FEEC0AF01C0E0C6E02C10BF0FEECDE
:1037C0000AF01D0E0C6E03C10BF0FEEC0AF000C1F6
:1037D00092F101C193F102C194F103C195F11FEF80
:1037E0001CF083C32AF184C32BF185C32CF186C35B
:1037F0002DF187C32EF188C32FF189C330F18AC31D
:1038000031F18CC332F18DC333F1010136EC2AF072
:10381000ADEC29F00101000E046F000E056F010EE2
:10382000066F000E076FFEEC28F000C192F101C197
:1038300093F102C194F103C195F11FEF1CF0160E34
:1038400015EC0BF0E8CF00F1170E15EC0BF0E8CFFC
:1038500001F1180E15EC0BF0E8CF02F1190E15EC82
:103860000BF0E8CF03F18BEC29F06EEC27F00401AC
:10387000730E826F57EC0EF004012C0E826F57EC22
:103880000EF08AC100F18BC101F18CC102F18DC132
:1038900003F18BEC29F06EEC27F00401730E826FBC
:1038A00057EC0EF004012C0E826F57EC0EF01A0E3E
:1038B00015EC0BF0E8CF00F11B0E15EC0BF0E8CF88
:1038C00001F11C0E15EC0BF0E8CF02F11D0E15EC0A
:1038D0000BF0E8CF03F145EC23F004012C0E826FCE
:1038E00057EC0EF092C100F193C101F194C102F1C5
:1038F00095C103F145EC23F061EC0EF02AEF23F0C3
:103900000401690E826F57EC0EF004012C0E826FD9
:1039100057EC0EF00101040E006F000E016F000E57
:10392000026F000E036F8BEC29F02CC182F40401AE
:10393000300E822757EC0EF02DC182F40401300EB8
:10394000822757EC0EF02EC182F40401300E82273C
:1039500057EC0EF02FC182F40401300E822757EC91
:103960000EF030C182F40401300E822757EC0EF0C5
:1039700031C182F40401300E822757EC0EF032C1BF
:1039800082F40401300E822757EC0EF033C182F42A
:103990000401300E822757EC0EF004012C0E826FCA
:1039A00057EC0EF00101060E006F000E016F000EC5
:1039B000026F000E036F8BEC29F02CC182F404011E
:1039C000300E822757EC0EF02DC182F40401300E28
:1039D000822757EC0EF02EC182F40401300E8227AC
:1039E00057EC0EF02FC182F40401300E822757EC01
:1039F0000EF030C182F40401300E822757EC0EF035
:103A000031C182F40401300E822757EC0EF032C12E
:103A100082F40401300E822757EC0EF033C182F499
:103A20000401300E822757EC0EF004012C0E826F39
:103A300057EC0EF001012B0E006F000E016F000E0F
:103A4000026F000E036F8BEC29F02CC182F404018D
:103A5000300E822757EC0EF02DC182F40401300E97
:103A6000822757EC0EF02EC182F40401300E82271B
:103A700057EC0EF02FC182F40401300E822757EC70
:103A80000EF030C182F40401300E822757EC0EF0A4
:103A900031C182F40401300E822757EC0EF032C19E
:103AA00082F40401300E822757EC0EF033C182F409
:103AB0000401300E822757EC0EF004012C0E826FA9
:103AC00057EC0EF0200EF86EF76AF66A0401090052
:103AD000F5CF82F457EC0EF00900F5CF82F457ECE5
:103AE0000EF00900F5CF82F457EC0EF00900F5CF87
:103AF00082F457EC0EF00900F5CF82F457EC0EF08B
:103B00000900F5CF82F457EC0EF00900F5CF82F4EE
:103B100057EC0EF00900F5CF82F457EC0EF061EC93
:103B20000EF02AEF23F08351630AD8A42AEF23F082
:103B30008451610AD8A42AEF23F085516C0AD8A4D5
:103B40002AEF23F08651410A3FE08651440A1BE0E8
:103B50008651420AD8B4F7EF1DF08651350AD8B421
:103B6000B4EF24F08651360AD8B409EF25F0865117
:103B7000370AD8B472EF25F08651380AD8B4D0EF9E
:103B800025F02AEF23F00798079A04017A0E826F36
:103B900057EC0EF00401780E826F57EC0EF0040122
:103BA000640E826F57EC0EF00401550E826F57ECD5
:103BB0000EF0E0EF1DF004014C0E826F57EC0EF09A
:103BC00061EC0EF02AEF23F00788079A04017A0EC1
:103BD000826F57EC0EF00401410E826F57EC0EF02D
:103BE0000401610E826F57EC0EF0D4EF1DF00798C0
:103BF000078A04017A0E826F57EC0EF00401420E20
:103C0000826F57EC0EF00401610E826F57EC0EF0DC
:103C1000D4EF1DF00101666715EF1EF0676715EF21
:103C20001EF0686715EF1EF0696715D04F6720EF2B
:103C30001EF0506720EF1EF0516720EF1EF0526714
:103C40000AD00101000E006F000E016F000E026F1E
:103C5000000E036F120011B80AD00101620E046F4A
:103C6000010E056F000E066F000E076F09D00101EF
:103C7000A70E046F020E056F000E066F000E076F91
:103C800066C100F167C101F168C102F169C103F1C8
:103C9000EDEC28F003BFBDEF1EF0119A119C01015D
:103CA000000E046FA80E056F550E066F020E076F0B
:103CB00066C100F167C101F168C102F169C103F198
:103CC00066C186F167C187F168C188F169C189F170
:103CD000EDEC28F003BF0BD00101000E866FA80E9B
:103CE000876F550E886F020E896F118A119C0E0E18
:103CF00015EC0BF0E8CF18F10F0E15EC0BF0E8CF38
:103D000019F1100E15EC0BF0E8CF1AF1110E15ECAD
:103D10000BF0E8CF1BF136EC28F086C104F187C127
:103D200005F188C106F189C107F1EDEC28F00782A1
:103D3000FAEC27F036EC28F00792FAEC27F086C16F
:103D400000F187C101F188C102F189C103F1079235
:103D5000FAEC27F0CC0E046FE00E056F870E066FAD
:103D6000050E076FEDEC28F000C118F101C119F143
:103D700002C11AF103C11BF13BD0119C119A010140
:103D8000800E006F1A0E016F060E026F000E036F99
:103D90004FC104F150C105F151C106F152C107F103
:103DA000EDEC28F003AF05D0E8EC29F0118C119A66
:103DB00012000E0E15EC0BF0E8CF18F10F0E15ECFB
:103DC0000BF0E8CF19F1100E15EC0BF0E8CF1AF15B
:103DD000110E15EC0BF0E8CF1BF14FC100F150C1F3
:103DE00001F151C102F152C103F10782FAEC27F04F
:103DF00018C100F119C101F11AC102F11BC103F18F
:103E000012000401730E826F57EC0EF004012C0EA9
:103E1000826F57EC0EF0078462C166F163C167F1EF
:103E200064C168F165C169F14BC14FF14CC150F1FA
:103E30004DC151F14EC152F157C159F158C15AF11A
:103E4000079427EC1FF061EC0EF02AEF23F066C117
:103E500000F167C101F168C102F169C103F101011B
:103E60008BEC29F06EEC27F00401630E826F57ECA7
:103E70000EF004012C0E826F57EC0EF04FC100F1D2
:103E800050C101F151C102F152C103F101018BECAA
:103E900029F06EEC27F00401660E826F57EC0EF0ED
:103EA00004012C0E826F57EC0EF0E8EC29F059C19A
:103EB00000F15AC101F101018BEC29F06EEC27F001
:103EC0000401740E826F57EC0EF012001082040190
:103ED000530E826F57EC0EF004012C0E826F57ECDC
:103EE0000EF083C32AF184C32BF185C32CF186C362
:103EF0002DF187C32EF188C32FF189C330F18AC316
:103F000031F18BC332F18CC333F1010136EC2AF06D
:103F1000ADEC29F000C166F101C167F102C168F1A1
:103F200003C169F18EC32AF18FC32BF190C32CF129
:103F300091C32DF192C32EF193C32FF194C330F1AD
:103F400095C331F196C332F197C333F1010136ECD9
:103F50002AF0ADEC29F000C14FF101C150F102C1CE
:103F600051F103C152F129EC2AF099C32FF19AC300
:103F700030F19BC331F19CC332F19DC333F1010198
:103F800036EC2AF0ADEC29F000C159F101C15AF12B
:103F900027EC1FF004012C0E826F57EC0EF0DAEFC5
:103FA0001FF018A001D0108C8251520A02E10F823A
:103FB00001D00F928251750A02E1108401D0109451
:103FC0008251550A02E1108601D0109611A003D04B
:103FD00011A401D01084078410B248EF20F010A47F
:103FE00034EF20F0B6C166F1B7C167F1B8C168F12E
:103FF000B9C169F1BAC16AF1BBC16BF1BCC16CF165
:10400000BDC16DF1BEC16EF1BFC16FF1C0C170F134
:10401000C1C171F1C2C172F1C3C173F1C4C174F104
:10402000C5C175F1C6C176F1C7C177F1C8C178F1D4
:10403000C9C179F1CAC17AF1CBC17BF1CCC17CF1A4
:10404000CDC17DF1CEC17EF1CFC17FF1D0C180F174
:10405000D1C181F1D2C182F1D3C183F1D4C184F144
:10406000D5C185F13CEF20F062C166F163C167F113
:1040700064C168F165C169F14BC14FF14CC150F1A8
:104080004DC151F14EC152F157C159F158C15AF1C8
:1040900007940FA06AEF20F00101926757EF20F01C
:1040A000936757EF20F0946757EF20F095675BEF29
:1040B00020F06AEF20F00AEC1EF092C104F193C1E7
:1040C00005F194C106F195C107F1EDEC28F003BFAD
:1040D000F0EF22F00AEC1EF00101000E046F000E5A
:1040E000056F010E066F000E076F1EEC29F011A080
:1040F0002CD011A22AD08BEC29F0296701D007D04F
:1041000004012D0E826F57EC0EF0EEEF22F030C15D
:1041100082F40401300E822757EC0EF031C182F494
:104120000401300E822757EC0EF032C182F40401F4
:10413000300E822757EC0EF033C182F40401300EAA
:10414000822757EC0EF0EEEF22F012A8C5D012989D
:1041500019C01AF01A3A1A42070E1A1600011A501C
:10416000000AD8B438EF21F000011A50010AD8B47F
:10417000C4EF20F000011A50020AD8B4C2EF20F0B8
:104180006AEF21F06AEF21F0E8EC29F029C001F193
:104190002AC000F1D89001330033D89001330033A6
:1041A0000101630E046F000E056F000E066F000E16
:1041B000076F1EEC29F0280E046F000E056F000E2D
:1041C000066F000E076FEDEC28F000C12CF0E8EC54
:1041D00029F027C001F1019F019D28C000F10101D4
:1041E000A40E046F000E056F000E066F000E076F21
:1041F0001EEC29F000C12BF000C104F101C105F152
:1042000002C106F103C107F1640E006F000E016FD9
:10421000000E026F000E036FEDEC28F0050E046F28
:10422000000E056F000E066F000E076F1EEC29F0E2
:1042300000C104F101C105F102C106F103C107F19A
:10424000E8EC29F02CC000F1EDEC28F000C12DF0D5
:104250002DC0E8FF050F2C5C03E78A846AEF21F08C
:104260002DC0E8FF0A0F2C5C01E68A946AEF21F06A
:1042700000C124F101C125F102C126F103C127F1DA
:10428000E8EC29F0EEEC29F019501F0BE8CF00F113
:104290000101640E046F000E056F000E066F000E24
:1042A000076FFEEC28F024C104F125C105F126C1F9
:1042B00006F127C107F1EDEC28F003BF02D08A9484
:1042C00001D08A8424C100F125C101F126C102F187
:1042D00027C103F1F0EF22F010AE4BD0109E00C1C9
:1042E00008F101C109F102C10AF103C10BF18BEC24
:1042F00029F030C1D6F131C1D7F132C1D8F133C183
:10430000D9F108C100F109C101F10AC102F10BC1E3
:1043100003F101016C0E046F070E056F000E066FAE
:10432000000E076FEDEC28F003BF04D00101550E1D
:10433000DA6F1CD008C100F109C101F10AC102F114
:104340000BC103F10101A40E046F060E056F000EF0
:10435000066F000E076FEDEC28F003BF04D00101DB
:104360007F0EDA6F03D00101FF0EDA6F1B8EF0EFC4
:1043700022F010A4C3EF21F00401750E826F57ECF8
:104380000EF0C8EF21F00401720E826F57EC0EF0B0
:1043900004012C0E826F57EC0EF08BEC29F029678C
:1043A000D7EF21F00401200E826FDAEF21F0040133
:1043B0002D0E826F57EC0EF030C182F40401300EE6
:1043C000822757EC0EF031C182F40401300E8227AF
:1043D00057EC0EF004012E0E826F57EC0EF032C136
:1043E00082F40401300E822757EC0EF033C182F4C0
:1043F0000401300E822757EC0EF004016D0E826F1F
:1044000057EC0EF004012C0E826F57EC0EF04FC1EA
:1044100000F150C101F151C102F152C103F101019A
:104420008BEC29F06EEC27F00401480E826F57ECFC
:104430000EF004017A0E826F57EC0EF004012C0E80
:10444000826F57EC0EF066C100F167C101F168C1DF
:1044500002F169C103F101018BEC29F06EEC27F048
:104460000401630E826F57EC0EF004012C0E826F74
:1044700057EC0EF066C100F167C101F168C102F1AD
:1044800069C103F101010A0E046F000E056F000EF1
:10449000066F000E076FFEEC28F0000E046F120E80
:1044A000056F000E066F000E076F1EEC29F08BECF7
:1044B00029F02AC182F40401300E822757EC0EF055
:1044C0002BC182F40401300E822757EC0EF02CC170
:1044D00082F40401300E822757EC0EF02DC182F4D5
:1044E0000401300E822757EC0EF02EC182F4040135
:1044F000300E822757EC0EF02FC182F40401300EEB
:10450000822757EC0EF030C182F40401300E82276E
:1045100057EC0EF004012E0E826F57EC0EF031C1F5
:1045200082F40401300E822757EC0EF032C182F47F
:104530000401300E822757EC0EF033C182F40401DF
:10454000300E822757EC0EF00401730E826F57EC89
:104550000EF004012C0E826F57EC0EF0E8EC29F0FF
:1045600059C100F15AC101F154EC24F00FB2BCEF73
:1045700022F00FA0EEEF22F004012C0E826F57EC18
:104580000EF0200EF86EF76AF66A04010900F5CF06
:1045900082F457EC0EF00900F5CF82F457EC0EF0E0
:1045A0000900F5CF82F457EC0EF00900F5CF82F444
:1045B00057EC0EF00900F5CF82F457EC0EF009002D
:1045C000F5CF82F457EC0EF00900F5CF82F457ECEA
:1045D0000EF00900F5CF82F457EC0EF061EC0EF00E
:1045E0000F902AEF23F00401630E826F57EC0EF058
:1045F00004012C0E826F57EC0EF030EC23F0040116
:104600002C0E826F57EC0EF0A3EC23F004012C0E5D
:10461000826F57EC0EF01FEC24F004012C0E826F19
:1046200057EC0EF00101F80E006FCD0E016F660E13
:10463000026F030E036F45EC23F004012C0E826F12
:1046400057EC0EF035EC24F061EC0EF02AEF23F07D
:1046500061EC0EF00301C26B0790109239EF26F067
:10466000D8900E0E15EC0BF0E8CF00F10F0E15EC04
:104670000BF0E8CF01F1100E15EC0BF0E8CF02F1D2
:10468000110E15EC0BF0E8CF03F10101000E046FE1
:10469000000E056F010E066F000E076F1EEC29F06D
:1046A0008BEC29F02AC182F40401300E822757ECEA
:1046B0000EF02BC182F40401300E822757EC0EF06D
:1046C0002CC182F40401300E822757EC0EF02DC16C
:1046D00082F40401300E822757EC0EF02EC182F4D2
:1046E0000401300E822757EC0EF02FC182F4040132
:1046F000300E822757EC0EF030C182F40401300EE8
:10470000822757EC0EF031C182F40401300E82276B
:1047100057EC0EF004012E0E826F57EC0EF032C1F2
:1047200082F40401300E822757EC0EF033C182F47C
:104730000401300E822757EC0EF004016D0E826FDB
:1047400057EC0EF01200120E15EC0BF0E8CF00F152
:10475000130E15EC0BF0E8CF01F1140E15EC0BF075
:10476000E8CF02F1150E15EC0BF0E8CF03F10101D3
:104770000A0E046F000E056F000E066F000E076F25
:10478000FEEC28F0000E046F120E056F000E066F8F
:10479000000E076F1EEC29F08BEC29F02AC182F481
:1047A0000401300E822757EC0EF02BC182F4040175
:1047B000300E822757EC0EF02CC182F40401300E2B
:1047C000822757EC0EF02DC182F40401300E8227AF
:1047D00057EC0EF02EC182F40401300E822757EC04
:1047E0000EF02FC182F40401300E822757EC0EF038
:1047F00030C182F40401300E822757EC0EF0040120
:104800002E0E826F57EC0EF031C182F40401300E8F
:10481000822757EC0EF032C182F40401300E822759
:1048200057EC0EF033C182F40401300E822757ECAE
:104830000EF00401730E826F57EC0EF012000A0E98
:1048400015EC0BF0E8CF00F10B0E15EC0BF0E8CFF8
:1048500001F10C0E15EC0BF0E8CF02F10D0E15EC8A
:104860000BF0E8CF03F154EF24F0060E15EC0BF03B
:10487000E8CF00F1070E15EC0BF0E8CF01F1080EC0
:1048800015EC0BF0E8CF02F1090E15EC0BF0E8CFB8
:1048900003F154EF24F00101E8EC29F0078457C13B
:1048A00000F158C101F107940101E80E046F800E78
:1048B000056F000E066F000E076FFEEC28F0000E6D
:1048C000046F040E056F000E066F000E076F1EECDE
:1048D00029F0880E046F130E056F000E066F000E90
:1048E000076FEDEC28F00A0E046F000E056F000E46
:1048F000066F000E076F1EEC29F08BEC29F001010A
:10490000296788EF24F00401200E826F8BEF24F0DA
:1049100004012D0E826F57EC0EF030C182F40401B9
:10492000300E822757EC0EF031C182F40401300EB4
:10493000822757EC0EF032C182F40401300E822738
:1049400057EC0EF004012E0E826F57EC0EF033C1BF
:1049500082F40401300E822757EC0EF00401430E5E
:10496000826F57EC0EF0120087C32AF188C32BF137
:1049700089C32CF18AC32DF18BC32EF18CC32FF187
:104980008DC330F18EC331F190C332F191C333F155
:104990000101296B36EC2AF0ADEC29F00101000E83
:1049A000046F000E056F010E066F000E076FFEEC20
:1049B00028F00E0E0C6E00C10BF0FEEC0AF00F0E8C
:1049C0000C6E01C10BF0FEEC0AF0100E0C6E02C171
:1049D0000BF0FEEC0AF0110E0C6E03C10BF0FEECB6
:1049E0000AF004017A0E826F57EC0EF004012C0ECF
:1049F000826F57EC0EF00401350E826F57EC0EF00B
:104A000004012C0E826F57EC0EF030EC23F0E0EF37
:104A10001DF087C32AF188C32BF189C32CF18AC307
:104A20002DF18BC32EF18CC32FF18DC330F18EC3CA
:104A300031F190C332F191C333F10101296B36ECAE
:104A40002AF0ADEC29F0880E046F130E056F000EEE
:104A5000066F000E076FF2EC28F0000E046F040ED4
:104A6000056F000E066F000E076FFEEC28F00101C7
:104A7000E80E046F800E056F000E066F000E076FC4
:104A80001EEC29F00A0E0C6E00C10BF0FEEC0AF0D1
:104A90000B0E0C6E01C10BF0FEEC0AF00C0E0C6E4E
:104AA00002C10BF0FEEC0AF00D0E0C6E03C10BF010
:104AB000FEEC0AF004017A0E826F57EC0EF004014E
:104AC0002C0E826F57EC0EF00401360E826F57ECFD
:104AD0000EF004012C0E826F57EC0EF01FEC24F048
:104AE000E0EF1DF087C32AF188C32BF189C32CF1B5
:104AF0008AC32DF18BC32EF18CC32FF18DC330F1FE
:104B00008FC331F190C332F191C333F1010136EC1F
:104B10002AF0ADEC29F0000E046F120E056F000EA6
:104B2000066F000E076FFEEC28F001010A0E046FFD
:104B3000000E056F000E066F000E076F1EEC29F0C9
:104B4000120E0C6E00C10BF0FEEC0AF0130E0C6E90
:104B500001C10BF0FEEC0AF0140E0C6E02C10BF05A
:104B6000FEEC0AF0150E0C6E03C10BF0FEEC0AF021
:104B700004017A0E826F57EC0EF004012C0E826F46
:104B800057EC0EF00401370E826F57EC0EF0040163
:104B90002C0E826F57EC0EF0A3EC23F0E0EF1DF02B
:104BA00087C32AF188C32BF189C32CF18AC32DF165
:104BB0008BC32EF18CC32FF18DC330F18EC331F135
:104BC00090C332F191C333F10101296B36EC2AF025
:104BD000ADEC29F0880E046F130E056F000E066F02
:104BE000000E076FF2EC28F0000E046F040E056F44
:104BF000000E066F000E076FFEEC28F00101E80EB4
:104C0000046F800E056F000E066F000E076F1EEC1E
:104C100029F0060E0C6E00C10BF0FEEC0AF0070E38
:104C20000C6E01C10BF0FEEC0AF0080E0C6E02C116
:104C30000BF0FEEC0AF0090E0C6E03C10BF0FEEC5B
:104C40000AF004017A0E826F57EC0EF004012C0E6C
:104C5000826F57EC0EF00401380E826F57EC0EF0A5
:104C600004012C0E826F57EC0EF035EC24F0E0EFCF
:104C70001DF007A8ADEF26F00101800E006F1A0E9F
:104C8000016F060E026F000E036F4BC104F14CC1A1
:104C900005F14DC106F14EC107F1EDEC28F003BF5F
:104CA000F4EF26F068EC27F04BC100F14CC101F1A4
:104CB0004DC102F14EC103F10782FAEC27F018C191
:104CC00004F119C105F11AC106F11BC107F1F80E73
:104CD000006FCD0E016F660E026F030E036FEDECD9
:104CE00028F00E0E0C6E00C10BF0FEEC0AF00F0E59
:104CF0000C6E01C10BF0FEEC0AF0100E0C6E02C13E
:104D00000BF0FEEC0AF0110E0C6E03C10BF0FEEC82
:104D10000AF007840101E8EC29F057C100F158C1FD
:104D200001F107940A0E0C6E00C10BF0FEEC0AF0C4
:104D30000B0E0C6E01C10BF0FEEC0AF00C0E0C6EAB
:104D400002C10BF0FEEC0AF00D0E0C6E03C10BF06D
:104D5000FEEC0AF00798F4EF26F007AAF4EF26F02D
:104D600007840101E8EC29F057C100F158C101F1B5
:104D70000794060E0C6E00C10BF0FEEC0AF0070E55
:104D80000C6E01C10BF0FEEC0AF0080E0C6E02C1B5
:104D90000BF0FEEC0AF0090E0C6E03C10BF0FEECFA
:104DA0000AF0078462C100F163C101F164C102F13C
:104DB00065C103F10794120E0C6E00C10BF0FEECFE
:104DC0000AF0130E0C6E01C10BF0FEEC0AF0140E8B
:104DD0000C6E02C10BF0FEEC0AF0150E0C6E03C156
:104DE0000BF0FEEC0AF0079A0401805181197F0B49
:104DF0000BE09EA809D014EE00F081517F0BE12654
:104E0000E750812B0F01AD6E05012F51010A13E010
:104E100081AA1BEF27F005012F51000A0AE00FB805
:104E20001BEF27F0050130671BEF27F00FB81BEFD2
:104E300027F08AEF30F081B830EF27F018EC2BF034
:104E400005012F51020A02E030EF27F05C2F30EF0E
:104E500027F05BC55CF50501010E306F3C0E316F2C
:104E6000ABEF0DF018C100F119C101F11AC102F147
:104E70001BC103F1000E046F000E056F010E066FDB
:104E8000000E076F1EEC29F029A15DEF27F02051DD
:104E9000D8B45DEF27F018C100F119C101F11AC1B2
:104EA00002F11BC103F1000E046F000E056F0A0E24
:104EB000066F000E076F1EEC29F01200010104516D
:104EC0000013055101130651021307510313120079
:104ED0000101186B196B1A6B1B6B12002AC182F44B
:104EE0000401300E822757EC0EF02BC182F404012E
:104EF000300E822757EC0EF02CC182F40401300EE4
:104F0000822757EC0EF02DC182F40401300E822767
:104F100057EC0EF02EC182F40401300E822757ECBC
:104F20000EF02FC182F40401300E822757EC0EF0F0
:104F300030C182F40401300E822757EC0EF031C1EB
:104F400082F40401300E822757EC0EF032C182F455
:104F50000401300E822757EC0EF033C182F40401B5
:104F6000300E822757EC0EF012002FC182F404019C
:104F7000300E822757EC0EF030C182F40401300E5F
:104F8000822757EC0EF031C182F40401300E8227E3
:104F900057EC0EF032C182F40401300E822757EC38
:104FA0000EF033C182F40401300E822757EC0EF06C
:104FB0001200060E1D6E060E1E6E060E1F6E1D2EB4
:104FC000DFEF27F01E2EDFEF27F01F2EDFEF27F099
:104FD0008B84020E1D6E020E1E6E020E1F6E1D2EA3
:104FE000EFEF27F01E2EEFEF27F01F2EEFEF27F049
:104FF0008B9412000101005305E1015303E10253B8
:1050000001E1002BBDEC28F0E8EC29F03951006FEC
:105010003A51016F420E046F4B0E056F000E066F82
:10502000000E076FFEEC28F000C104F101C105F18C
:1050300002C106F103C107F118C100F119C101F164
:105040001AC102F11BC103F107B22BEF28F0F2ECF9
:1050500028F02DEF28F0EDEC28F000C118F101C187
:1050600019F102C11AF103C11BF11200E8EC29F099
:1050700059C100F15AC101F1060E15EC0BF0E8CF51
:1050800004F1070E15EC0BF0E8CF05F1080E15EC56
:105090000BF0E8CF06F1090E15EC0BF0E8CF07F1A5
:1050A000EDEC28F000C124F101C125F102C126F187
:1050B00003C127F1290E046F000E056F000E066F65
:1050C000000E076FFEEC28F0EE0E046F430E056F26
:1050D000000E066F000E076FF2EC28F024C104F1F9
:1050E00025C105F126C106F127C107F1FEEC28F024
:1050F00000C11CF101C11DF102C11EF103C11FF16C
:10510000120E15EC0BF0E8CF04F1130E15EC0BF0BA
:10511000E8CF05F1140E15EC0BF0E8CF06F1150EF3
:1051200015EC0BF0E8CF07F10D0E006F000E016FCC
:10513000000E026F000E036FFEEC28F0180E046FD5
:10514000000E056F000E066F000E076F1EEC29F0B3
:105150001CC104F11DC105F11EC106F11FC107F1FB
:10516000F2EC28F06A0E046F2A0E056F000E066F2F
:10517000000E076FEDEC28F01200BF0EFA6E200E45
:105180003A6F396BD8900037013702370337D8B000
:10519000CEEF28F03A2FC3EF28F039073A07035330
:1051A000D8B412000331070B80093F6F03390F0B8E
:1051B000010F396F80EC5FF0406F390580EC5FF0D4
:1051C000405D405F396B3F33D8B0392739333FA951
:1051D000E3EF28F040513927120001010DEC2AF0CD
:1051E000D8B01200010103510719346FD0EC29F037
:1051F000D8900751031934AF800F12000101346BAE
:10520000F4EC29F0D8A00AEC2AF0D8B01200DFECB8
:1052100029F0E8EC29F01F0E366F20EC2AF00B3550
:10522000D8B0D0EC29F0D8A00335D8B01200362F72
:105230000DEF29F034B1F7EC29F012000101346BC5
:1052400004510511061107110008D8A0F4EC29F04B
:10525000D8A00AEC2AF0D8B01200086B096B0A6BD0
:105260000B6B20EC2AF01F0E366F20EC2AF0075152
:105270000B5DD8A448EF29F006510A5DD8A448EF89
:1052800029F00551095DD8A448EF29F00451085DC3
:10529000D8A05BEF29F00451085F0551D8A0053D67
:1052A000095F0651D8A0063D0A5F0751D8A0073D07
:1052B0000B5FD8900081362F35EF29F034B1F7EC31
:1052C00029F0346BF4EC29F0D89024EC2AF0075143
:1052D0000B5DD8A478EF29F006510A5DD8A478EFC9
:1052E00029F00551095DD8A478EF29F00451085D33
:1052F000D8A087EF29F0003F87EF29F0013F87EF23
:1053000029F0023F87EF29F0032BD8B4120034B103
:10531000F7EC29F012000101346BF4EC29F0D8B05D
:10532000120029EC2AF0200E366F003701370237C1
:10533000033711EE33F00A0E376FE7360A0EE75CDB
:10534000D8B0E76EE552372F9DEF29F0362F95EF55
:1053500029F034B12981D890120001010A0E346F6E
:10536000200E366F11EE29F03451376F0A0ED890A7
:10537000E652D8B0E726E732372FB8EF29F00333EB
:10538000023301330033362FB2EF29F0E750FF0F1D
:10539000D8A00335D8B0120029B1F7EC29F01200DB
:1053A000045100270551D8B0053D01270651D8B05A
:1053B000063D02270751D8B0073D032712000051D0
:1053C000086F0151096F02510A6F03510B6F1200F0
:1053D0000101006B016B026B036B12000101046B96
:1053E000056B066B076B12000335D8A01200035142
:1053F000800B001F011F021F031F003F07EF2AF051
:10540000013F07EF2AF0023F07EF2AF0032B342B6E
:10541000032512000735D8A012000751800B041F86
:10542000051F061F071F043F1DEF2AF0053F1DEF54
:105430002AF0063F1DEF2AF0072B342B0725120018
:105440000037013702370337083709370A370B3778
:1054500012000101296B2A6B2B6B2C6B2D6B2E6BB1
:105460002F6B306B316B326B336B120001012A51A1
:105470000F0B2A6F2B510F0B2B6F2C510F0B2C6F17
:105480002D510F0B2D6F2E510F0B2E6F2F510F0B18
:105490002F6F30510F0B306F31510F0B316F325175
:1054A0000F0B326F33510F0B336F120010A806D061
:1054B0008994000EC76E220EC66E05D08984000E38
:1054C000C76E220EC66E050EE82EFED7120010A87B
:1054D00002D0898401D08994050EE82EFED71200EF
:1054E00056EC2AF09E96C69E000EC96EFF0E9EB622
:1054F00002D0E82EFCD79E96C69E000EC96EFF0E07
:105500009EB602D0E82EFCD7C9CFABF59E96C69EBC
:10551000000EC96EFF0E9EB602D0E82EFCD7C9CF92
:10552000ACF59E96C69E000EC96EFF0E9EB602D0CA
:10553000E82EFCD7C9CFADF59E96C69E000EC96E6B
:10554000FF0E9EB602D0E82EFCD7C9CFAEF59E96D0
:10555000C69E000EC96EFF0E9EB602D0E82EFCD786
:10556000C9CFAFF59E96C69E000EC96EFF0E9EB6C1
:1055700002D0E82EFCD7C9CFB0F59E96C69E000E8D
:10558000C96EFF0E9EB602D0E82EFCD7C9CFB1F58A
:1055900067EC2AF0120056EC2AF09E96C69E800E0A
:1055A000C96EFF0E9EB602D0E82EFCD79E96C69E10
:1055B000ABC5C9FFFF0E9EB602D0E82EFCD79E9663
:1055C000C69EACC5C9FFFF0E9EB602D0E82EFCD722
:1055D0009E96C69EADC5C9FFFF0E9EB602D0E82EB0
:1055E000FCD79E96C69EAEC5C9FFFF0E9EB602D0E2
:1055F000E82EFCD79E96C69EAFC5C9FFFF0E9EB68D
:1056000002D0E82EFCD79E96C69EB0C5C9FFFF0EFD
:105610009EB602D0E82EFCD79E96C69EB1C5C9FFA5
:10562000FF0E9EB602D0E82EFCD767EC2AF01200DF
:1056300056EC2AF09E96C69E070EC96EFF0E9EB6C9
:1056400002D0E82EFCD79E96C69E000EC96EFF0EB5
:105650009EB602D0E82EFCD7C9CFABF59E96C69E6B
:10566000000EC96EFF0E9EB602D0E82EFCD7C9CF41
:10567000ACF59E96C69E000EC96EFF0E9EB602D079
:10568000E82EFCD7C9CFADF59E96C69E000EC96E1A
:10569000FF0E9EB602D0E82EFCD7C9CFAEF567EC60
:1056A0002AF056EC2AF09E96C69E21C0C9FFFF0E36
:1056B0009EB602D0E82EFCD79E96C69E000EC96EFE
:1056C000FF0E9EB602D0E82EFCD7C9CFB2F567EC2C
:1056D0002AF0120056EC2AF09E96C69E870EC96EDE
:1056E000FF0E9EB602D0E82EFCD79E96C69EABC596
:1056F000C9FFFF0E9EB602D0E82EFCD79E96C69E2E
:10570000ACC5C9FFFF0E9EB602D0E82EFCD79E9610
:10571000C69EADC5C9FFFF0E9EB602D0E82EFCD7CF
:105720009E96C69EAEC5C9FFFF0E9EB602D0E82E5D
:10573000FCD767EC2AF056EC2AF09E96C69E22C053
:10574000C9FFFF0E9EB602D0E82EFCD79E96C69EDD
:10575000B2C5C9FFFF0E9EB602D0E82EFCD767EC9B
:105760002AF0120056EC2AF09E96C69E870EC96E4D
:10577000FF0E9EB602D0E82EFCD79E96C69E000E67
:10578000C96EFF0E9EB602D0E82EFCD79E96C69E2E
:10579000800EC96EFF0E9EB602D0E82EFCD79E96F4
:1057A000C69E800EC96EFF0E9EB602D0E82EFCD7B4
:1057B0009E96C69E800EC96EFF0E9EB602D0E82E43
:1057C000FCD767EC2AF0120056EC2AF09E96C69E93
:1057D000870EC96EFF0E9EB602D0E82EFCD79E96AD
:1057E000C69E000EC96EFF0E9EB602D0E82EFCD7F4
:1057F0009E96C69E000EC96EFF0E9EB602D0E82E83
:10580000FCD79E96C69E800EC96EFF0E9EB602D035
:10581000E82EFCD79E96C69E800EC96EFF0E9EB6E1
:1058200002D0E82EFCD767EC2AF0120010A82DD089
:1058300056EC2AF09E96C69E22C0C9FFFF0E9EB669
:1058400002D0E82EFCD79E96C69E450EC96EFF0E6E
:105850009EB602D0E82EFCD767EC2AF056EC2AF070
:105860009E96C69E8F0EC96EFF0E9EB602D0E82E83
:10587000FCD79E96C69E000EC96EFF0E9EB602D045
:10588000E82EFCD767EC2AF0120056EC2AF09E9620
:10589000C69E22C0C9FFFF0E9EB602D0E82EFCD7DE
:1058A0009E96C69E010EC96EFF0E9EB602D0E82ED1
:1058B000FCD767EC2AF056EC2AF09E96C69E910E15
:1058C000C96EFF0E9EB602D0E82EFCD79E96C69EED
:1058D000A50EC96EFF0E9EB602D0E82EFCD767EC6F
:1058E0002AF0120056EC2AF09E96C69E22C0C9FFEE
:1058F000FF0E9EB602D0E82EFCD79E96C69E810E65
:10590000C96EFF0E9EB602D0E82EFCD767EC2AF0D7
:10591000120056EC2AF09E96C69E22C0C9FFFF0ECA
:105920009EB602D0E82EFCD79E96C69E010EC96E8A
:10593000FF0E9EB602D0E82EFCD767EC2AF01200CC
:1059400056EC2AF09E96C69E910EC96EFF0E9EB62C
:1059500002D0E82EFCD79E96C69EA50EC96EFF0EFD
:105960009EB602D0E82EFCD767EC2AF0120056EC67
:105970002AF09E96C69E910EC96EFF0E9EB602D06C
:10598000E82EFCD79E96C69E000EC96EFF0E9EB6F0
:1059900002D0E82EFCD767EC2AF012000501256B37
:1059A000266B276B286B899A400EC76E200EC66E39
:1059B0009E96C69E030EC96EFF0E9EB602D0E82EBE
:1059C000FCD79E96C69E27C5C9FFFF0E9EB602D085
:1059D000E82EFCD79E96C69E26C5C9FFFF0E9EB632
:1059E00002D0E82EFCD79E96C69E25C5C9FFFF0EA5
:1059F0009EB602D0E82EFCD79E96C69EC952FF0ED8
:105A00009EB602D0E82EFCD7898A0F01C950FF0A42
:105A100001E1120005012E51130A05E005012E5186
:105A2000170A0CE012000501F00E256FFF0E266F1D
:105A30000F0E276F000E286F27EF2DF00501F00ED7
:105A4000256FFF0E266FFF0E276F000E286F899AB5
:105A5000400EC76E200EC66E9E96C69E030EC96E81
:105A6000FF0E9EB602D0E82EFCD79E96C69E27C596
:105A7000C9FFFF0E9EB602D0E82EFCD79E96C69EAA
:105A800026C5C9FFFF0E9EB602D0E82EFCD79E9613
:105A9000C69E25C5C9FFFF0E9EB602D0E82EFCD7D4
:105AA0009E96C69EC952FF0E9EB602D0E82EFCD727
:105AB000898A0F01C950FF0A1DE005012E51130A02
:105AC00005E005012E51170A0BE012000501000E3A
:105AD000256F000E266F100E276F000E286F120024
:105AE0000501000E256F000E266F000E276F010EB8
:105AF000286F12000501256B266B276B286B0501AB
:105B00002E51130A05E005012E51170A0CE0120070
:105B10000501000E216F000E226F080E236F000E8C
:105B2000246F9CEF2DF00501000E216F000E226FF7
:105B3000800E236F000E246F21C500F122C501F1F4
:105B400023C502F124C503F125C504F126C505F1DD
:105B500027C506F128C507F15EEC27F000C125F541
:105B600001C126F502C127F503C128F5899A400E27
:105B7000C76E200EC66E9E96C69E030EC96EFF0EA1
:105B80009EB602D0E82EFCD79E96C69E27C5C9FFBA
:105B9000FF0E9EB602D0E82EFCD79E96C69E26C566
:105BA000C9FFFF0E9EB602D0E82EFCD79E96C69E79
:105BB00025C5C9FFFF0E9EB602D0E82EFCD79E96E3
:105BC000C69EC952FF0E9EB602D0E82EFCD7898A27
:105BD000C950FF0A08E104C125F505C126F506C133
:105BE00027F507C128F5D890050124332333223344
:105BF00021332151F00B216F216706EF2EF0226730
:105C000006EF2EF0236706EF2EF024679CEF2DF0B1
:105C10000501100E2527E86A2623E86A2723E86A8B
:105C200028231200E86A05012E51130A06E0050137
:105C30002E51170A0BE0020E120005012851000A2E
:105C400003E12751F00B07E0010E12000501285176
:105C5000000A01E0010E120029C500F12AC501F178
:105C60002BC502F12CC503F125C504F126C505F1AC
:105C700027C506F128C507F1EDEC28F003BF120097
:105C800012EC2EF0D8A4A4EF2EF0899A400EC76E25
:105C9000200EC66E9E96C69E060EC96EFF0E9EB65E
:105CA00002D0E82EFCD7898A899A9E96C69E020E5B
:105CB000C96EFF0E9EB602D0E82EFCD79E96C69EF9
:105CC00027C5C9FFFF0E9EB602D0E82EFCD79E96D0
:105CD000C69E26C5C9FFFF0E9EB602D0E82EFCD791
:105CE0009E96C69E25C5C9FFFF0E9EB602D0E82E21
:105CF000FCD79E96C69E000EC96EFF0E9EB602D0C1
:105D0000E82EFCD7898A899A9E96C69E050EC96E92
:105D1000FF0E9EB602D0E82EFCD79E96C69EC952B4
:105D2000FF0E9EB602D0E82EFCD7C9B08DEF2EF044
:105D3000898A0501100E2527E86A2623E86A2723A9
:105D4000E86A28232CEF2EF01200899A400EC76EC5
:105D5000200EC66E9E96C69E060EC96EFF0E9EB69D
:105D600002D0E82EFCD7898A899A9E96C69EC70ED5
:105D7000C96EFF0E9EB602D0E82EFCD7898A0501B7
:105D8000256B266B276B286B1200899A400EC76E15
:105D9000200EC66E9E96C69E050EC96EFF0E9EB65E
:105DA00002D0E82EFCD79E96C69EC952FF0E9EB624
:105DB00002D0E82EFCD7C9CF33F5898A1200899A20
:105DC000400EC76E200EC66E9E96C69EB90EC96E58
:105DD000FF0E9EB602D0E82EFCD7898A1200899A5F
:105DE000400EC76E200EC66E9E96C69EAB0EC96E46
:105DF000FF0E9EB602D0E82EFCD7898AFF0EE82E51
:105E0000FED7120012EC2EF0D8A41200899A400E90
:105E1000C76E200EC66E9E96C69E030EC96EFF0EFE
:105E20009EB602D0E82EFCD79E96C69E27C5C9FF17
:105E3000FF0E9EB602D0E82EFCD79E96C69E26C5C3
:105E4000C9FFFF0E9EB602D0E82EFCD79E96C69ED6
:105E500025C5C9FFFF0E9EB602D0E82EFCD79E9640
:105E6000C69EC952FF0E9EB602D0E82EFCD7898A84
:105E70000F01C950FF0AD8A4FDEF2FF00501FE0E57
:105E8000336F70EC2AF0ABC534F5ACC535F5ADC554
:105E900036F5AEC537F5AFC538F5B0C539F5B1C57E
:105EA0003AF50784B6C166F1B7C167F1B8C168F1C8
:105EB000B9C169F14BC14FF14CC150F14DC151F124
:105EC0004EC152F157C159F158C15AF10AEC1EF0B6
:105ED00000C13BF501C13CF502C13DF503C13EF5F2
:105EE00005015D677BEF2FF05E677BEF2FF05F674B
:105EF0007BEF2FF060677FEF2FF08CEF2FF05DC509
:105F000004F15EC505F15FC506F160C507F1EDEC72
:105F100028F003BFFDEF2FF059C13FF55AC140F5FE
:105F2000B5C541F5B6C542F507940501110E326FAE
:105F3000899A400EC76E200EC66E9E96C69E060EAD
:105F4000C96EFF0E9EB602D0E82EFCD7898A899AC8
:105F50009E96C69E020EC96EFF0E9EB602D0E82E19
:105F6000FCD79E96C69E27C5C9FFFF0E9EB602D0DF
:105F7000E82EFCD79E96C69E26C5C9FFFF0E9EB68C
:105F800002D0E82EFCD79E96C69E25C5C9FFFF0EFF
:105F90009EB602D0E82EFCD725EE33F0322F02D089
:105FA000DDEF2FF09E96C69EDECFC9FFFF0E9EB698
:105FB00002D0E82EFCD7CEEF2FF0898A899A9E96E0
:105FC000C69E050EC96EFF0E9EB602D0E82EFCD707
:105FD0009E96C69EC952FF0E9EB602D0E82EFCD7F2
:105FE000C9B0E8EF2FF0898A0501100E2527E86A6D
:105FF0002623E86A2723E86A2823120021C500F136
:1060000022C501F123C502F124C503F1899A400E8E
:10601000C76E200EC66E9E96C69E0B0EC96EFF0EF4
:106020009EB602D0E82EFCD79E96C69E02C1C9FF3E
:10603000FF0E9EB602D0E82EFCD79E96C69E01C1EA
:10604000C9FFFF0E9EB602D0E82EFCD79E96C69ED4
:1060500000C1C9FFFF0E9EB602D0E82EFCD79E9667
:10606000C69EC952FF0E9EB602D0E82EFCD725EE82
:1060700033F00501100E326F9E96C69EC952FF0E78
:106080009EB602D0E82EFCD7C9CFDEFF322F3CEF00
:1060900030F0898A1200899A400EC76E200EC66EB3
:1060A0009E96C69E900EC96EFF0E9EB602D0E82E3A
:1060B000FCD79E96C69E000EC96EFF0E9EB602D0FD
:1060C000E82EFCD79E96C69E000EC96EFF0E9EB6A9
:1060D00002D0E82EFCD79E96C69E000EC96EFF0E1B
:1060E0009EB602D0E82EFCD79E96C69EC952FF0EE1
:1060F0009EB602D0E82EFCD7C9CF2DF59E96C69E3F
:10610000C952FF0E9EB602D0E82EFCD7C9CF2EF59D
:10611000898A1200D9EC27F0B5C5E8FFD70802E359
:10612000D9EC27F0B5C5E8FFC80802E3D9EC27F0A1
:10613000B5C5E8FFB90802E3D9EC27F0B5C5E8FF1B
:10614000AA0802E3D9EC27F0B5C5E8FF9B0802E3F3
:10615000D9EC27F018EC2BF0DFEC2EF0F29CF29E3D
:106160008B94C69AC2909482948C720ED36ED3A4F0
:10617000FED789968A909390FF0EE8CF00F0E82E24
:10618000FED7002EFCD78150F294F29A9E909D90FB
:106190009E929D92F298F292F290F286F28E030015
:0261A000FF00FE
:10BF0000E844F926000C160C2B0C3F0C520C640C68
:10BF1000760C860C960CA50CB30CC10CCF0CDC0C6B
:06BF2000E80CF40C000C1B
:0200000400F00A
:0100C800FE39
:00000001FF
